:02000000E52FEA
:10080C007630472CF0002225F100080064008001AE
:10081C00840A04060319003404060D2C83120511F6
:10082C008514182C192C1A2C1B2C83120515080056
:10083C0083120515212C222C232C242C8312851495
:10084C00272C282C292C2A2C831285102D2C2E2C6D
:10085C002F2C302C0800831205158514352C362CC2
:10086C00372C382C831205113B2C3C2C3D2C3E2C68
:10087C0083128510412C422C432C442C08007030E0
:10088C00472C831687008D3083129E00F8309F0012
:10089C0083168C0105141C141B14831205101F10D5
:1008AC008F118E118E130800831205115D2C5E2C96
:1008BC005F2C602C83128514632C642C652C662CA5
:1008CC0083128510692C6A2C6B2C6C2C83120515E9
:1008DC00080083128514831605158312051D792CC7
:1008EC00F101F10A7A2CF10183160511831205111D
:1008FC000630F000F00B802C000083128510862C43
:10090C00872C882C892C71080800F001831605159A
:10091C00F1010310F00D83128514942C952C962C58
:10092C00972C83120519F00A85109C2C9D2C9E2C5B
:10093C009F2C0830F10A7102031C902C83160511B0
:10094C0070080800F500F601740876020318C42C30
:10095C00142431247508C5246F24003A031DC42CBB
:10096C007208C5246F24003A031DC42C7308C524D7
:10097C006F24003A031DC42CF60AAA2C142CF00088
:10098C00F101F01FCC2C83120515CE2C831205110E
:10099C00CF2CD02CD12CD22C83128514D52CD62C28
:1009AC00D72CD82C8312851007307106031905112A
:1009BC000310F00DE12CE22CE32CE42C0830F10AAE
:1009CC00710203180800C72CF2002F308316950013
:1009DC007208900083120F1320301B2522309100D7
:1009EC0083120F1FF62C8530F100F10BFB2C7208D3
:1009FC0083169000013091000F0A031D042D70081E
:100A0C008F0083120F1310301B25123091008312AC
:100A1C000F1F0D2D1A30F100F10B122D0000720872
:100A2C0022257006031908001A2D83169100163022
:100A3C009200F13092000800831690000130910072
:100A4C000F080800F60031247608C5246F24003AFC
:100A5C00031D6B2D7208C5246F24003A031D6B2DEA
:100A6C00312476080138C5246F24003A031D6B2D00
:100A7C0083160515F701F8017808803AF4008030E8
:100A8C007402031D4B2D7308770203186B2D8B24F6
:100A9C008312AF0083160511532D542D552D562D51
:100AAC007308FF3EF400FF3003180030F5007806A1
:100ABC00031D622D770874060319662D5A24672DC1
:100ACC001E24F70A0319F80A422D142C0530AB0129
:100ADC0008248312B500FB303502031C7A2D053037
:100AEC00F001EA248312B5010A3035020318F72D00
:100AFC0004303506031DAA2DE127EA24DC27640007
:100B0C000330FB000830FA007730F900F90B8C2D1C
:100B1C00FA0B8C2DFB0B8C2D831206100330FB0073
:100B2C000830FA007730F900F90B9A2DFA0B9A2D50
:100B3C00FB0B9A2D831206140330FD0A7D02031C55
:100B4C00852DAB01AB0AF72D09303506031DE42DBD
:100B5C000530F001EA24DC2764000330FB00083088
:100B6C00FA007730F900F90BB92DFA0BB92DFB0B04
:100B7C00B92D831206100330FB000830FA007730D1
:100B8C00F900F90BC72DFA0BC72DFB0BC72D8312E0
:100B9C0006140530FD0A7D02031CB22D64000330DF
:100BAC00FB000830FA007730F900F90BDB2DFA0B5B
:100BBC00DB2DFB0BDB2D83120614D42D0A303502F2
:100BCC000318B501E127EA240B30FB002630FA00AC
:100BDC005D30F900F90BF02DFA0BF02DFB0BF02D1D
:100BEC00F72D8316061485100511051485111C1498
:100BFC001B141E141D14FC011330F2009B30D12762
:100C0C00A8240D30F900F90B092E1330F200E23054
:100C1C00F301F30A28250D30F900F90B132E0530DA
:100C2C00FC0A7C02031C022E2330F2000C30D1276C
:100C3C00A8242430F2000330D127A8240430F20079
:100C4C002030D127A8240B30F2002230D127A82441
:100C5C001030F2002030D127A8240A30F2004030A6
:100C6C00D127A8240330F2004030D127A8241C300F
:100C7C00F2002130D127A8241A30F2004530D127B8
:100C8C00A8241B30F2000430D127A8242B081830DC
:100C9C00F2000319652E8030D127A8241930D627ED
:100CAC00A8241D30D627A8241E30F2007730D12777
:100CBC00A8241F30F200E230F301F30A772EC03083
:100CCC00D127A8241930D627A8241D30D627A8242C
:100CDC001E30F200FA30D127A8241F30F200E23087
:100CEC00F301F401F40AA8242030D627A8242130DB
:100CFC00F200FA30D127A8242230D627A8241530A8
:100D0C00FB004B30FA00BE30F900F90B8B2EFA0BBE
:100D1C008B2EFB0B8B2E00000530F001EA242930C2
:100D2C00FB009630FA007F30F900F90B9B2EFA0B82
:100D3C009B2EFB0B9B2E83128F118E118E13640036
:100D4C0003308312A501A50AFB000830FA007730A6
:100D5C00F900F90BAF2EFA0BAF2EFB0BAF2E0630B2
:100D6C00FA003030F900F90BB92EFA0BB92E00004D
:100D7C0083122B080319C62E831606146400C42E86
:100D8C00AA01AA0AA001A101A9015A2F2A08031D30
:100D9C00152F8E13831606140630FA003030F90026
:100DAC00F90BD62EFA0BD62E000083120608A600DD
:100DBC00261CF42E8E13A501A50AA4012C08031DD4
:100DCC005A2F0530AC01AC0A08248312B500350843
:100DDC0003195A2F0530F001EA245A2F0B30A40ABC
:100DEC002402031C5A2F1830A401A501A801A80A3B
:100DFC00AE01AD01A301A201F2008030D127A824DD
:100E0C001930F200FE30D127A8240630FA00303019
:100E1C00F900F90B0F2FFA0B0F2F00005A2F8E131E
:100E2C00831606148530F900F90B1A2F8312060865
:100E3C00A600261C2A2F8E13A501A50AA401A90120
:100E4C00A90AA001A1015A2FA00A0319A10A8530F1
:100E5C00F900F90B2F2F8312290803193B2F0B30A4
:100E6C00A40A2402031C5A2F442F273021021130CC
:100E7C0003192002031C5A2FA001A1011830F20003
:100E8C008030D127A8241930F200FE30D127A824B5
:100E9C000630FA003030F900F90B522FFA0B522FB2
:100EAC0000008312AA01A401640083122508031D0B
:100EBC00CC2E06248530F900F90B622F8312A70182
:100ECC00A2018312280803195A2F64008530F900F7
:100EDC00F90B6E2F831227080319C52F1F1C922F95
:100EEC000A30A201A30A2302031C672FA301AE013F
:100EFC002D08031D672F1830AD01AD0AF200FF302D
:100F0C00D127A8241930F200EF30D127A82485303E
:100F1C00F900F90B8F2F672F0A30A301A20A2202C6
:100F2C00031C672FA201AD012E08031D672F18307B
:100F3C00AE01AE0AF2008030D127A8241930D62792
:100F4C00A8241D30D627A8241E30F200A630D127A5
:100F5C00A8241F30F2000E30D127A8243430FA0018
:100F6C00F130F900F90BB82FFA0BB82FBD2F831203
:100F7C008E13A501A50AA401A801AA018D2F1F1883
:100F8C00662F0B30A20A2202031C672FA201A701B5
:100F9C00A70A4524672FF300E230F401F40A080095
:100FAC00F200E230F301F401F40A080006101E14FA
:100FBC001D14FD010800B50A3508F0000534A130F8
:100FCC00B000A030B1000130B2000430B300E23008
:100FDC00B40020308313840030300C2483016C2D3A
:06400000E33F5D3FF03FCD
:00000001FF
